:04000000C5EF10F048
:1000080000C01EF001C01DF002C01CF003C01BF0B0
:1000180004C01AF005C019F008C018F009C017F09C
:100028000AC016F00BC015F0E1CF27F0E2CF28F098
:10003800E9CF25F0EACF26F0F3CF23F0F4CF24F070
:10004800F5CF22F0F8CF1FF0F7CF20F0F6CF21F050
:100058009EAA44D09DAA42D0ACA203D0AC98AC884A
:10006800AC92ACA402D0AFCF71F1AFCF71F1010166
:1000780071510D0A07E0000E735D02E1500E725DCA
:1000880001E21ED0010E0B6F000E0C6F000E735DA7
:1000980002E1500E725D04E3020E0B6F000E0C6F4E
:1000A800A09A0F0E7225E16E010E7321E26EE66AC8
:1000B80072C174F173C175F1726B736B716B0ED091
:1000C8000F0E7225E16E010E7321E26E71C1E6FF1B
:1000D80072C174F173C175F1724B732BA4AA44D029
:1000E800A3AA42D09CA203D09C989C889C929CA4D2
:1000F80002D0AACF00F10101AACF00F100510D0AE8
:1001080007E0000E045D02E1500E035D01E21ED01F
:10011800010E4F6E000E506E000E045D02E1500E8F
:10012800035D04E3020E4F6E000E506EA09AAF0EF0
:100138000325E16E000E0421E26EE66A03C109F1AF
:1001480004C10AF1036B046B006B0ED0AF0E0325DC
:10015800E16E000E0421E26E00C1E6FF03C109F161
:1001680004C10AF1034B042BF2AA15D0F2A413D050
:100178000101924B932B000E006E9351005C02E13B
:100188009251090807E2010E016F000E026FF29A00
:10019800926B936BF294D1EC0DF022C0F5FF1FC067
:1001A800F8FF20C0F7FF21C0F6FF23C0F3FF24C0EB
:1001B800F4FF1EC000F01DC001F01CC002F01BC0FF
:1001C80003F01AC004F019C005F018C008F017C0F1
:1001D80009F016C00AF015C00BF025C0E9FF26C0CB
:0C01E800EAFF27C0E1FF28C0E2FF110081
:1001F4001E0E0F014D6F100E01017C6F040E7D6FFA
:100204007CC1E1FF7DC1E2FFE69E7CC1E1FF7DC1CF
:10021400E2FFE69C040E7C25E16E000E7D21E26E79
:10022400E68C180E966F040E976F96C1E1FF97C186
:10023400E2FFE69E96C1E1FF97C1E2FFE69C040E51
:100244009625E16E000E9721E26EE68C020E7C2567
:10025400E16E000E7D21E26EA1C1E6FFA2C1E6FFC0
:10026400010E7C25E16E000E7D21E26E400EE66EED
:100274007CC1E9FF7DC1EAFFEECF00F07CC1E1FF64
:100284007DC1E2FF400E0014E66E7CC1E9FF7DC132
:10029400EAFFEECF00F07CC1E1FF7DC1E2FF880EF2
:1002A4000010E66E7CC1ACF17DC1ADF1040E7C1989
:0802B400006E00C07CF1120095
:1002BC000B6A0A6A096A00500402F4CF09F0F3CF02
:1002CC0008F001500502F4CF0BF0F3CF0AF0005008
:1002DC000502F3500926F4500A22E86A0B22015059
:1002EC000402F3500926F4500A22E86A0B2208C0D3
:1002FC0000F009C001F00AC002F00BC003F01200BC
:10030C0004012251010A13E120C401F01F0E011651
:10031C000150000A0CE10101A78F04012151030ACD
:10032C0004E1010E01018A6F02D001018A6B040104
:10033C002251000AD8A48DD020C401F01F0E011642
:10034C000150020AD8A485D024C401F00F0E011666
:10035C000150000AD8B47DD00101A78F040124BF3D
:10036C0016D024C403F00F0E031603C000F0000EC9
:10037C00016E0036009001367A0E0024E96E010EF3
:10038C000120EA6EEECF04F0EECF05F015D024C4B8
:10039C0003F00F0E031603C000F0000E016E0036C2
:1003AC0000900136940E0024E96E010E0120EA6ED5
:1003BC00EECF04F0EECF05F02151030A07E104C0A3
:1003CC00E1FF05C0E2FF840EE66E43D024C400F0CA
:1003DC000F0E00164C0E026E0F0E036E005002260E
:1003EC00D8B0032A02C0E9FF03C0EAFFFE0EEE14E8
:1003FC00006EEECF01F0FF0E011602C0E1FF03C04C
:10040C00E2FF00C0E6FF01C0E6FF24AF11D004C03C
:10041C00E1FF05C0E2FFE66A040E0418006E00C09E
:10042C0004F004C0E1FF05C0E2FF400EE66E11D0FF
:10043C0004C0E1FF05C0E2FF880EE66E040E04184E
:10044C00006E00C004F004C0E1FF05C0E2FFC80E5E
:04045C00E66E120036
:100460000401286B296B4AD00101A78F0401288160
:1004700001018A51010A02E10401288354D00101DB
:10048000A78F51D00101A78F040124BF16D024C427
:1004900003F00F0E031603C000F0000E016E0036CD
:1004A000009001367A0E0024E96E010E0120EA6EFA
:1004B000EECF04F0EECF05F015D024C403F00F0EFC
:1004C000031603C000F0000E016E003600900136E6
:1004D000940E0024E96E010E0120EA6EEECF04F0C6
:1004E000EECF05F004C0E9FF05C0EAFFEECF01F052
:1004F00001A403D00401010E286F15D020C401F01F
:100500001F0E01160150000AAFE020C401F01F0EBB
:1005100001160150010AB3E020C401F01F0E0116BC
:100520000150020AAFE00101A7AF07D0280EA46F67
:0C053000040EA56FA781020EA86F120038
:10053C00000E0101A95D02E1080EA85D10E2A8C140
:10054C0003F0A9C104F0A351000A03E1010EA36F4B
:10055C0005D0A351010A02E1020EA36F04D0080ECC
:10056C00036E000E046E94C1E1FF95C1E2FFE692AA
:10057C0094C1E1FF95C1E2FFE69094C1E9FF95C1FA
:10058C00EAFFEECF00F094C1E1FF95C1E2FF045009
:10059C000010E66E010E9425E16E000E9521E26EC0
:1005AC0003C0E6FF0350A85D006E0450A959016E0C
:1005BC0000C0A8F101C0A9F1280E8B6F040E8C6F3E
:1005CC00A7B12FD0035004102BE0A4C1F6FFA5C196
:1005DC00F7FFA6C1F8FF0900F5CF00F08BC1E1FFD2
:1005EC008CC1E2FF00C0E6FF8B4B8C2B010EA425C7
:1005FC00006E000EA521016E000EA621026E00C039
:10060C00A4F101C0A5F102C0A6F1010E035C006EBD
:10061C00000E0458016E00C003F001C004F0D2D7E4
:10062C0024D00350041021E0A4C1E9FFA5C1EAFFC6
:10063C008BC1E1FF8CC1E2FFEECFE6FF8B4B8C2B25
:10064C00010EA425006E000EA521016E00C0A4F1C0
:10065C0001C0A5F1010E035C006E000E0458016E82
:0C066C0000C003F001C004F0DCD7120055
:1006780020C401F01F0E01160150010A01E094D0B8
:1006880004012451000A01E08FD02151060A42E1F9
:1006980037D00101AA51010A17E1150E006E280E84
:1006A800016E000E026E120E0026000E01220222BA
:1006B80000C0A4F101C0A5F102C0A6F1090EA86FFF
:1006C800000EA96FC00EA76F25D00101AA51010A1B
:1006D80012E1FA0E006E280E016E000E026E00C0C6
:1006E800A4F101C0A5F102C0A6F1210EA86F000E69
:1006F800A96FC00EA76F0ED00101800EA76F0AD098
:1007080004012351210AC5E02351220ADEE02351C6
:10071800230AF2E020C401F0600E0116050E006EF7
:10072800005004E00132019EFF0FFBD70150010A7F
:1007380001E03AD026D038D037D0890E0101A46F15
:10074800010EA56F010EA86F000EA96FC10EA76F4D
:100758002BD00101800EA76F23C489F125D0010198
:10076800880EA46F010EA56F010EA86F000EA96F69
:10077800810EA76F19D00101800EA76F22C488F1DE
:1007880013D004012151010AD6E02151090AD4E00D
:100798002151020AD2E021510A0ADBE02151030A61
:0A07A800DEE021510B0AE7E0120029
:1007B2000101A78F0F014D6B0101796B22C4AAF1D0
:1007C200AA51000A03E1100EAB6F03D0200EAB6FEB
:0407D20010DD120024
:1007D60004012051800AD8A478D0C00E0101A76F69
:1007E60069D00101D70E006E290E016E000E026E51
:1007F60000C0A4F101C0A5F102C0A6F1120EA86FB7
:10080600000EA96F62D00101030E006E000E016E8C
:1008160022C404F0000E056E4EDD610E0024E96E62
:10082600010E0120EA6EEECFA4F1EECFA5F1EECFD8
:10083600A6F1020EA425F66E000EA521F76E000E97
:10084600A621F86E0900F5CF00F00900F5CF01F0FA
:1008560000C0A8F101C0A9F138D00401225101015C
:10086600825D23E3030E006E000E016E22C404F0C7
:10087600000E056E20DD680E0024E96E010E0120D3
:10088600EA6EEECFA4F1EECFA5F1EECFA6F1A4C1AC
:10089600F6FFA5C1F7FFA6C1F8FF0900F5CF00F0E6
:1008A60000C0A8F1000EA96F01D0A76B0ED0010100
:1008B600A76B0BD004012351010A93E02351020ACE
:0C08C600A2E02351030AC9E0F2D712009F
:1008D20020C401F0600E0116050E006E005004E007
:1008E2000132019EFF0FFBD70150000A01E05ED0EA
:1008F2003AD00101A78F080EAB6F58D06BDF56D0EC
:1009020057DF54D00101AA0EA46F010EA56FA78173
:10091200010EA86FA78F4AD0A2DD48D0F6DC46D0E0
:10092200790E006E010E016E040124510026D8B02A
:10093200012A00C0A4F101C0A5F10101A781010EA5
:10094200A86FA78F33D00101A78F790EE16E010E38
:10095200E26E04012451E126D8B0E22A22C4E6FF65
:1009620025D024D023D004012151050AC2E021510F
:10097200060AC4E02151090AC3E02151080AC2E073
:100982002151000AC9E02151010AC8E02151030A9C
:10099200C5E021510A0AC4E021510B0AD4E02151D9
:0E09A200070ADFE021510C0ADDE0DCD712006D
:1009B000160E0F015F6F9F0E5D6F3B0E5C6F120096
:1009C00065980101A7BF4BD09AAF2AD0020E000153
:1009D000FF6F010E01019425E16E000E9521E26E7C
:1009E000E66A94C1E1FF95C1E2FFC80EE66E010E12
:1009F0008E25E16E000E8F21E26E080EE66E020E6D
:100A00008E25E16E000E8F21E26E280EE66E040E3A
:100A1000E66E8EC1E1FF8FC1E2FFC80EE66E1ED00A
:100A2000010E8E25E16E000E8F21E26E080EE66E3D
:100A3000020E8E25E16E000E8F21E26E200EE66E14
:100A4000040EE66E8EC1E1FF8FC1E2FF8C0EE66EF2
:100A500094C1E1FF95C1E2FF840EE66E85D09ABF96
:100A600083D0040120AF57D00101A9510401275DB3
:100A700004E10101A8510401265D04E226C4A8F1A5
:100A800027C4A9F15BDD010E0001FF6F010E01011A
:100A90008E25E16E000E8F21E26E080EE66E020ECC
:100AA0008E25E16E000E8F21E26E200EE66E040EA2
:100AB000E66E8EC1E1FF8FC1E2FF800EE66E8D6BA8
:100AC000010E9025E16E000E9121E26E080EE66E99
:100AD000020E9025E16E000E9121E26E200EE66E70
:100AE000040EE66E90C1E1FF91C1E2FF840EE66E56
:100AF000010E8D6F020E9425E16E000E9521E26EBF
:100B0000280EE66E040EE66E94C1E1FF95C1E2FF89
:100B1000C80EE66E29D0020E0001FF6F010E010122
:100B20009425E16E000E9521E26EE66A94C1E1FF24
:100B300095C1E2FFC80EE66E010E8E25E16E000E35
:100B40008F21E26E080EE66E020E8E25E16E000E1B
:100B50008F21E26E280EE66E040EE66E8EC1E1FF76
:0A0B60008FC1E2FFC80EE66E12001E
:0A0B6A000101785301E083DD120061
:100B7400150E0101616F280E626F000E636F7F0E08
:100B8400686F2A0E696F000E6A6FD60E6B6F280E9F
:100B94006C6F000E6D6FE70E6E6F270E6F6F000E99
:040BA400706F12005C
:100BA8000001FF6B94C1E1FF95C1E2FFE66A040E04
:100BB80001019419E16E95C1E2FF000EE21AE66A9E
:080BC8009AAF01D09A9F1200C0
:100BD000010E01019025E96E000E9121EA6EEECF23
:100BE00000F000C002F0000E9C5D02E102509B5D2F
:100BF00003E29BC102F00AD002509B5D006E000E22
:100C00009C59016E00C09BF101C09CF1036A025027
:100C1000035C1CE2280EE96E040EEA6E0350E9261E
:100C2000D8B0EA2AEECF00F098C1E1FF99C1E2FF07
:100C300000C0E6FF010E9825006E000E9921016E9E
:100C400000C098F101C099F1032AE1D7000E006EAF
:100C50009C51005C02E19B51000828E2010E8E25A8
:100C6000E16E000E8F21E26E080EE66E020E8E25FA
:100C7000E16E000E8F21E26E280EE66E040EE66E27
:100C800090C1E9FF91C1EAFFEECF00F000BC07D0B0
:100C90008EC1E1FF8FC1E2FFC80EE66E06D08EC1A5
:100CA000E1FF8FC1E2FF880EE66E19D0010E8E259E
:100CB000E16E000E8F21E26E080EE66E020E8E25AA
:100CC000E16E000E8F21E26E200EE66E040EE66EDF
:100CD0008EC1E1FF8FC1E2FF840EE66E9A9F120083
:100CE00065920F015C9562A403D0FB0E6216FBD7E0
:020CF0001200F0
:100CF20040DFAC6BAD6B7E6B7F6B636A626A57DE03
:100D0200658C5E6B4D6B659C0101806B816B000E87
:100D1200815D02E1080E805D17E280C100F081C1B1
:100D220001F0003600900136003600900136000EC8
:100D32000024E16E040E0120E26EE66AE66AE66ACB
:100D4200E66A804B812BE3D7160E0F014C6F62A629
:100D520003D0F70E6216FBD70101A76B9A6B9B6B50
:100D62009C6B6598080E946F040E956FAA6BAB6B23
:020D720012006D
:100D74000F014CA119D090C1E9FF91C1EAFFEECF58
:100D840001F00150800A0FE194C1E9FF95C1EAFF27
:100D9400EECF01F00150840A06E190C1E1FF91C158
:0E0DA400E2FF8C0EE66E4C91DF0E621612001E
:040DB200A1981200F2
:100DB60094C1E9FF95C1EAFFEECF00F000AE05D081
:100DC60094C1E1FF95C1E2FFE66A0101A36B000150
:100DD600FF6B0101A86BA96BA76B78DDC3DEEDDDA8
:020DE6001200F9
:100DE8000001FF51020A02E1EFDE1ED0D9DE8D516B
:100DF800000A19E1010E8E25E16E000E8F21E26EC8
:100E0800080EE66E020E8E25E16E000E8F21E26E50
:100E1800200EE66E040EE66E8EC1E1FF8FC1E2FF82
:0A0E28008C0EE66E01D08D6B1200F7
:0C0E32000F015C85EF0E62166582120055
:100E3E00040E01019419006E00C094F1AB51080A22
:100E4E000DE122C45EFF0F015E51000804E2100E98
:100E5E000101AB6F03D00101040EAB6F0001FF5116
:100E6E00010A3CE1020E01019425E16E000E95216E
:100E7E00E26E280EE66E040EE66E9EEC02F0A351B4
:100E8E00020A07E194C1E1FF95C1E2FF840EE66E0E
:100E9E0024D0040E9419006E00C094F194C1E9FFA1
:100EAE0095C1EAFFEECF00F000BC0CD0040E9419F1
:100EBE00006E00C094F194C1E1FF95C1E2FFC80E2F
:100ECE00E66E0BD0040E9419006E00C094F194C11E
:100EDE00E1FF95C1E2FF880EE66E01D05EDE1200E4
:100EEE00000E0101C61902E1000EC51902E1016AE8
:100EFE000AD0C5C1E9FFC6C1EAFFEECF00F0000E71
:0C0F0E0000BE010E016E01C000F01200D8
:100F1A000101AB51000A0BE1656A0F015C6B43DD0D
:100F2A0065B602D06586FCD7010E0101AB6FAB51E5
:100F3A00010A0AE165BA08D0626A0F015C6B5C813A
:100F4A005C89020E0101AB6F62A406D00F015CA599
:100F5A0003D0FB0E6216BFDE65A202D025DFDCD00D
:100F6A0062A019D00F015CA116D0BEDE040EAB6FD1
:100F7A00200E0401026F040E036F080E016F000EAB
:100F8A000015006E00C000F48C0E0011006E00C047
:100F9A0000F4FE0E621662A806D00F015CA903D007
:100FAA0043DFEF0E621662AC05D00F015CAD02D0D2
:100FBA00BF0E621662AA04D00F015CAB01D0D5DE67
:100FCA0062A204D00F015CA301D0636A040E01017E
:100FDA00AB5D02E2E9DEA0D00F015CA79CD0010163
:100FEA00C66B040EC65DD8B096D062A691D064CF07
:100FFA0083F1F70E6216780E8315016E0150000A0E
:10100A00D8A485D0FD0E8315016E026AFF0E021662
:10101A00000E021802E1000E01186BE17E0E831524
:10102A00016E01C003F00332039E03C000F0000EFC
:10103A00016E003600900136003600900136000E2F
:10104A000024026E040E0120036E02C090F103C058
:10105A0091F102C08EF103C08FF1040E8E19006E59
:10106A0000C08EF102C0E9FF03C0EAFFEECF00F034
:10107A0000C001F03C0E01160132019E0132019EB0
:10108A0001500D0A34E1020E9025E96E000E9121FD
:10109A00EA6EEECF01F0EECF02F00250040A02E14E
:1010AA00280E011822E1020E9025E16E000E912110
:1010BA00E26E200EE66E040EE66EC56B080EC55D86
:1010CA0014E2200EE16E040EE26EC551E126D8B09C
:1010DA00E22A280EE96E040EEA6EC551E926D8B056
:1010EA00EA2AEECFE6FFC52BE9D760DE01D077DE2C
:1010FA000DD0FD0E8315016E026AFF0E0216000E58
:10110A00021802E1040E011801E194DE00D001D0B8
:0A111A0002D0C62B66D748DE120093
:101124000101C651000A12E0C5C100F0000E016EB3
:10113400003600900136940E0024E96E010E012061
:10114400EA6EEECF04F0EECF05F011D0C5C100F089
:10115400000E016E0036009001367A0E0024E96E0E
:10116400010E0120EA6EEECF04F0EECF05F0020E80
:101174000424E16E000E0520E26EC7C1E6FFC8C17B
:10118400E6FF010E0424E16E000E0520E26EC9C1E3
:10119400E6FF04C0E9FF05C0EAFFEECF00F004C09B
:1011A400E1FF05C0E2FF400E0014E66E04C0E9FF53
:1011B40005C0EAFFEECF00F004C0E1FF05C0E2FF86
:1011C400880E0010E66EC651000A1BE0C5C100F08F
:1011D400000E016E003600900136940E0024026E5B
:1011E400010E0120036E02C0E9FF03C0EAFF040EF2
:1011F400EE18006E02C0E1FF03C0E2FF00C0E6FF8C
:101204001AD0C5C100F0000E016E00360090013600
:101214007A0E0024026E010E0120036E02C0E9FF63
:1012240003C0EAFF040EEE18006E02C0E1FF03C023
:10123400E2FF00C0E6FF04C000F005C001F01200A8
:0A124400D08EA288A088F28E12005E
:10124E000101C26BC36BC46B020EBF25F66E000E9E
:10125E00C021F76E000EC121F86E0900F5CF05F022
:10126E00030EBF25F66E000EC021F76E000EC121D3
:10127E00F86E0900F5CF00F000C003F0000E046E0A
:10128E0003C001F0006A05500024066E000E012016
:10129E00076EBFC108F0C0C109F0C1C10AF0010E4E
:1012AE000824F66E000E0920F76E000E0A20F86E66
:1012BE000900F5CF01F00150020A1BE1060E0824C9
:1012CE00F66E000E0920F76E000E0A20F86E090069
:1012DE00F5CF01F00150C25D0CE2060E0824F66E49
:1012EE00000E0920F76E000E0A20F86E0900F5CFE9
:1012FE00C2F1010E0824F66E000E0920F76E000EE4
:10130E000A20F86E0900F5CF01F00150040A1BE126
:10131E00080E0824F66E000E0920F76E000E0A2045
:10132E00F86E0900F5CF01F00150C25D0CE2080E17
:10133E000824F66E000E0920F76E000E0A20F86ED5
:10134E000900F5CFC2F108C0F6FF09C0F7FF0AC0C9
:10135E00F8FF0900F5CF00F00050C325016E000E16
:10136E00C421026E01C0C3F102C0C4F10750025C79
:10137E0002E10650015C01E30FD008C0F6FF09C080
:10138E00F7FF0AC0F8FF0900F5CF00F0005008265D
:0E139E00000E09220A2283D7C2C100F01200FD
:1013AC00200E0101AB5D03E365B201D002D0006AEF
:1013BC0046D07EC1C5F17FC1C6F193DD00523EE13E
:1013CC00C2C1C5F1010EC66FBFC1C7F1C0C1C8F122
:1013DC00C1C1C9F1A1DE00C07EF101C07FF1846BF7
:1013EC00856B866B876B7EC1C5F17FC1C6F179DDDC
:1013FC0000520FE0010E016E0150000A01E187DD81
:10140C000101845185118611871102E0006A17D001
:10141C00EAD77EC1C3F17FC1C4F1000E7F1902E18E
:10142C00000E7E1909E0010EC325E96E000EC421E1
:10143C00EA6EEECF00F003D0006A01D0006A120011
:10144C00D70E006E290E016E000E026E0E0E0024D9
:10145C00F66E000E0120F76E000E0220F86E0900E9
:10146C00F5CF03F003C004F00F0E0024F66E000E4F
:10147C000120F76E000E0220F86E0900F5CF01F086
:10148C000150035C12E2D70E006E290E016E000EA5
:10149C00026E0F0E0024F66E000E0120F76E000E89
:1014AC000220F86E0900F5CF04F0D70E006E290E5D
:1014BC00016E000E026E100E0024F66E000E01205E
:1014CC00F76E000E0220F86E0900F5CF01F0015006
:1014DC00045C12E2D70E006E290E016E000E026E35
:1014EC00100E0024F66E000E0120F76E000E022086
:0E14FC00F86E0900F5CF04F004C000F01200F5
:10150A00086A096A100E0C6E01340836093604504E
:10151A00085E0550D8A0053C095ED8B007D0045033
:10152A0008260550D8B0053C0926D8900036013661
:06153A000C2EEAD712009E
:0E154000A8B202D00000FCD7B8C1A9FF12006B
:10154E000B6A0A6A096A086A0E6A0334083604507E
:10155E00085E0550D8A0053C095E0650D8A0063C92
:10156E000A5E0750D8A0073C0B5EE86AD8A0010EB1
:10157E000E5E0336070E0C6E0334083609360A3635
:10158E000B360E36045003A012D0085E0550D8A0BC
:10159E00053C095E0650D8A0063C0A5E0750D8A04E
:1015AE00073C0B5EE86AD8A0010E0E5E11D008262D
:1015BE000550D8B0053C09260650D8B0063C0A2680
:1015CE000750D8B0073C0B26E86AD8B0010E0E269D
:1015DE0003360C2ED1D70234083609360A360B36AE
:1015EE000E36045003A012D0085E0550D8A0053C5C
:1015FE00095E0650D8A0063C0A5E0750D8A0073CEC
:10160E000B5EE86AD8A0010E0E5E11D008260550BA
:10161E00D8B0053C09260650D8B0063C0A2607501D
:10162E00D8B0073C0B26E86AD8B0010E0E2602365B
:10163E00070E0C6E0234083609360A360B360E3695
:10164E00045002A012D0085E0550D8A0053C095ED9
:10165E000650D8A0063C0A5E0750D8A0073C0B5E89
:10166E00E86AD8A0010E0E5E11D008260550D8B03B
:10167E00053C09260650D8B0063C0A260750D8B0BD
:10168E00073C0B26E86AD8B0010E0E2602360C2E49
:10169E00D1D70134083609360A360B360E360450C9
:1016AE0002A012D0085E0550D8A0053C095E065077
:1016BE00D8A0063C0A5E0750D8A0073C0B5EE86A2D
:1016CE00D8A0010E0E5E11D008260550D8B0053CEC
:1016DE0009260650D8B0063C0A260750D8B0073C5B
:1016EE000B26E86AD8B0010E0E260136070E0C6ED8
:1016FE000134083609360A360B360E36045001A070
:10170E0012D0085E0550D8A0053C095E0650D8A040
:10171E00063C0A5E0750D8A0073C0B5EE86AD8A0CC
:10172E00010E0E5E11D008260550D8B0053C0926D4
:10173E000650D8B0063C0A260750D8B0073C0B26F8
:10174E00E86AD8B0010E0E2601360C2ED1D7003421
:10175E00083609360A360B360E36045001A012D062
:10176E00085E0550D8A0053C095E0650D8A0063C80
:10177E000A5E0750D8A0073C0B5EE86AD8A0010E9F
:10178E000E5E11D008260550D8B0053C092606502D
:10179E00D8B0063C0A260750D8B0073C0B26E86A9C
:1017AE00D8B0010E0E260036070E0C6E0034083629
:1017BE0009360A360B360E36045000A012D0085EDB
:1017CE000550D8A0053C095E0650D8A0063C0A5E1E
:1017DE000750D8A0073C0B5EE86AD8A0010E0E5E3B
:1017EE0011D008260550D8B0053C09260650D8B0B1
:1017FE00063C0A260750D8B0073C0B26E86AD8B03C
:10180E00010E0E2600360C2ED1D700B00ED004508D
:10181E0008260550D8B0053C09260650D8B0063C1F
:0C182E000A260750D8B0073C0B26120019
:0E183A00ADB202D00000FCD7B8C1AEFF120064
:101848000101BE6B200EAB5D03E365B201D002D08F
:10185800006A2ED0ACC1C5F1ADC1C6F177EC07F076
:10186800005225E1ACC1BCF1ADC1BDF1000EAD190E
:1018780002E1000EAC190AE0010EBC25E96E000E6B
:10188800BD21EA6EEECF00F000C0BEF1BBC1C5F1CC
:10189800C66BB8C1C7F1B9C1C8F1BAC1C9F13EDC5C
:1018A80000C0ACF101C0ADF1BEC100F001D0006ACA
:0218B80012001C
:1018BA00C8DD00C0B8F1150E0101BF6F280EC06F58
:1018CA00000EC16FBFDC00C0B9F1B851005C03E281
:0C18DA00B8C100F002D0B9C100F012004B
:0E18E600570E0D6E0D2EFED7000000001200F2
:1018F400B8C1BFF1B9C1C0F1BAC1C1F1010E010152
:06190400C26F52DD12006B
:10190A000101AB51000A0DE1656A0F015C6BD8EC6D
:10191A0004F093DC65B602D06586FCD7010E01019E
:04192A00AB6F12008D
:10192E00D596D584D592D590D59AD59C6D0ED76E79
:10193E00840ED66EF2940101926B936B016B026B67
:08194E00F184F28AD58E12002B
:10195600B1DF00C082F1010E786FAEC1A1F1AFC157
:10196600A2F1B0C176F1B1C177F179EC06F0010EC2
:0C197600016E0150010A01E1C5DF120002
:101982003A0E516E180E526EB80E536E010E546E10
:10199200FF0E476EFF0E486E000E496E000E4A6E35
:1019A200FF0E4B6EFF0E4C6E000E4D6E000E4E6E15
:1019B200FF0E0101056FFF0E066F000E076F000E8E
:1019C200086FAD8A900EAC6E948E949C9EAA03D042
:0819D200AFCF00F0FBD71200BB
:1019DA000101B46BB56B000EB55D02E10A0EB45D90
:1019EA000BE2B451B225E16EB551B321E26E200E7D
:1019FA00E66EB44BB52BEFD7B451B225E16EB551B3
:101A0A00B321E26EE66A010EB45F000EB55BB45113
:101A1A00B225B66FB551B321B76F0A0E046E000E28
:101A2A00056E066E076EAEC100F0AFC101F0B0C11F
:101A3A0002F0B1C103F086DD08C000F009C001F070
:101A4A000AC002F00BC003F0300E0026B6C1E1FF57
:101A5A00B7C1E2FF00C0E6FF0A0E046E000E056E73
:101A6A00066E076EAEC100F0AFC101F0B0C102F060
:101A7A00B1C103F067DD00C0AEF101C0AFF102C031
:101A8A00B0F103C0B1F1000E046E031808E104506E
:101A9A00021805E10450011802E10050000A01E1B0
:0E1AAA0005D0010EB45F000EB55BB1D712007F
:101AB8000900F5CFE6FF0006FBE10106F9E1120097
:101AC800AF0E01010325E16E000E0421E26EE66A05
:101AD800096B0A6B036B046BAACF00F1006B4F6AAA
:061AE800506AA08A120002
:101AEE00400E516E150E526EB80E536E010E546EA0
:101AFE00FF0E476EFF0E486E000E496E000E4A6EC8
:101B0E00FF0E4B6EFF0E4C6E000E4D6E000E4E6EA7
:101B1E00FF0E0101056FFF0E066F000E076F000E20
:101B2E00086FA88A900E9C6E98849892A4AA03D0EF
:081B3E00AACF00F0FBD7120052
:101B4600AEC1F6FFAFC1F7FFB0C1F8FF0900F5CF90
:101B560000F0005211E0AEC1F6FFAFC1F7FFB0C111
:101B6600F8FF0900F5CFB8F165DE010E0101AE27D9
:0A1B7600000EAF23B023E4D71200E5
:101B8000FE0EC16EFF0EC26EFF0E926EFF0E946EC1
:101B9000FF0E986E958E9986959896988C988D984C
:021BA000120031
:101BA2000101AB51010A09E165BA07D0626A0F016E
:101BB2005C815C89020E0101AB6F62A407D00F0148
:101BC2005CA504D0FB0E621670EC06F065A203D091
:101BD200D9EC06F0E4D062A01AD00F015CA117D0B4
:101BE20079EC06F0040EAB6F200E0401026F040EB6
:101BF200036F080E016F000E0015006E00C000F4A6
:101C02008C0E0011006E00C000F4FE0E621662A877
:101C120007D00F015CA904D019EC07F0EF0E621691
:101C220062AC05D00F015CAD02D0BF0E621662AA93
:101C320005D00F015CAB02D0BAEC06F062A204D070
:101C42000F015CA301D0636A040E0101AB5D03E2E4
:101C5200D9EC06F0A4D00F015CA79FD00101CB6B99
:101C6200040ECB5DD8B099D062A694D064CF83F134
:101C7200F70E6216780E8315016E0150000AD8A481
:101C820088D0FD0E8315016E026AFF0E0216000E49
:101C9200021802E1000E01186DE17E0E8315016E3D
:101CA20001C003F00332039E03C000F0000E016E78
:101CB200003600900136003600900136000E0024F6
:101CC200026E040E0120036E02C090F103C091F176
:101CD20002C08EF103C08FF1040E8E19006E00C097
:101CE2008EF102C0E9FF03C0EAFFEECF00F000C0B0
:101CF20001F03C0E01160132019E0132019E01509B
:101D02000D0A35E1020E9025E96E000E9121EA6E70
:101D1200EECF01F0EECF02F00250040A02E1280EEB
:101D2200011822E1020E9025E16E000E9121E26E71
:101D3200200EE66E040EE66ECA6B080ECA5D14E251
:101D4200200EE16E040EE26ECA51E126D8B0E22AFC
:101D5200280EE96E040EEA6ECA51E926D8B0EA2AC4
:101D6200EECFE6FFCA2BE9D7DBEC06F002D0F4ECAB
:101D720006F00ED0FD0E8315016E026AFF0E0216EA
:101D8200000E021802E1040E011802E11FEC07F036
:101D920000D001D002D0CB2B63D7D9EC06F01200D1
:101DA2008C988D981F0E0B6E710E0C6E1E0E0D6EA2
:101DB2000D2EFED70C2EFCD70B2EFAD700008C88E6
:101DC2001F0E0B6E710E0C6E1E0E0D6E0D2EFED7BB
:101DD2000C2EFCD70B2EFAD700008C988D881F0E84
:101DE2000B6E710E0C6E1E0E0D6E0D2EFED70C2E8E
:101DF200FCD70B2EFAD700008C888D981F0E0B6E25
:101E0200710E0C6E1E0E0D6E0D2EFED70C2EFCD713
:0C1E12000B2EFAD700008C988D9812005F
:101E1E000D0E0501406F0A0E416F426B400E01011F
:101E2E00B86F050EB96F400EBA6F5DDD005201E15D
:041E3E00F5D71200C2
:101E42000D0E0101B86FA0EC0AF00A0E0101B86F85
:061E5200A0EC0AF01200F2
:101E5800800E006EBB0E016E000E026E036E120045
:101E68000D0E0101B86FE5DC0A0E0101B86FE1DC67
:021E7800120056
:101E7A000101B26B050EB25D0AE2B251B025E16E04
:101E8A00000EB121E26E200EE66EB22BF3D7B251EC
:101E9A00B025E16E000EB121E26EE66AB207B251D8
:101EAA00B025B36F000EB121B46F0A0E046E000E96
:101EBA00056EAEC100F0AFC101F085EC0AF008C0B2
:101ECA0000F009C001F0300E0026B3C1E1FFB4C131
:101EDA00E2FF00C0E6FF0A0E046E000E056EAEC1F8
:101EEA0000F0AFC101F085EC0AF000C0AEF101C00C
:101EFA00AFF1000E011802E1000E001801E102D054
:061F0A00B207CDD7120062
:101F1000C26A070EC16EC18EAEC100F000360090DD
:101F2000003600900050C212C280DDDCC282C2A224
:101F300001D0FDD7C4CF01F0006AC3500012000EDB
:061F40000112C290120024
:101F4600AEC102F0AFC103F002C000F003C001F061
:101F5600024A032A00C0E9FF01C0EAFFEE5201E08F
:101F6600F3D70101AE51025C006EAF510358016E0A
:0A1F7600010E005E000E015A120079
:101F80000101B16BAEC1E9FFAFC1EAFFEECFB0F125
:101F9000B051000A0EE0B0C1B8F14FDC0101B12B25
:101FA000B151AE25E96E000EAF21EA6EEECFB0F171
:041FB000EFD7120055
:101FB400B2C100F00101B207005228E0AEC1E9FF4E
:101FC400AFC1EAFFEE50000A0CE0AEC1E9FFAFC1B9
:101FD400EAFFB0C1D9FFB1C1DAFFEE50DE1801E16A
:101FE4000FD0AEC1E9FFAFC1EAFFB0C1D9FFB1C1A3
:101FF400DAFFDE50EE5C006E016A000E015A08D072
:102004000101AE4BAF2BB04BB12BD2D7006A016AA2
:022014001200B8
:10201600AEC1F6FFAFC1F7FFB0C1F8FF0900F5CFBB
:1020260000F0005212E0AEC1F6FFAFC1F7FFB0C13B
:10203600F8FF0900F5CFB8F1A0EC0AF0010E010196
:0C204600AE27000EAF23B023E3D712003A
:10205200C29EC29CC29AC298C296C294C280010E0B
:10206200C26EC18EC19CC18AC188C196C182C1841F
:04207200C190120007
:10207600B0C1F6FFB1C1F7FFB2C1F8FF0900F5CF55
:1020860000F0005218E0B0C1F6FFB1C1F7FFB2C1CF
:10209600F8FF0900F5CF00F0AEC1E1FFAFC1E2FFE6
:1020A60000C0E6FF0101AE4BAF2B010EB027000EBC
:1020B600B123B223DDD7AEC1E1FFAFC1E2FFE66ACD
:0220C600120006
:1020C800AEC104F0AFC105F004C002F005C003F0D2
:1020D800044A052AB0C100F0B1C101F00101B04BBA
:1020E800B12B00C0E9FF01C0EAFF02C0E1FF03C055
:1020F800E2FFEECFE6FF02C0E9FF03C0EAFFEE52BF
:0E21080001E0E2D7AEC100F0AFC101F012005D
:102116000F0E01017225E16E010E7321E26EE66A71
:10212600746B756B726B736BAFCF71F1716B0B6BFD
:062136000C6BA08A1200F0
:10213C000101B16BAEC1E9FFAFC1EAFFEECFB0F167
:10214C00B051000A0FE0B0C1B8F1A0EC0AF00101E7
:10215C00B12BB151AE25E96E000EAF21EA6EEECF78
:06216C00B0F1EED71200F5
:10217200A1C1B8F1A2C1B9F1400E0101BA6F010EBD
:08218200BB6F24EC0CF012000D
:10218A0042EC15F0F8DC08DE6D0E0001AD6F000EB2
:10219A00AE6F6D6B556A7E86020E7F6E700EB06EE4
:1021AA00AD84C1EC0CF00C0EB86F1DEC0CF01F0ED8
:1021BA000B6E710E0C6E1E0E0D6E0D2EFED70C2EB2
:1021CA00FCD70B2EFAD70000390E0101AE6F290E8B
:1021DA00AF6F000EB06FB2DCB90E0101AE6F270E01
:1021EA00AF6F000EB06FAADC4E0E0101AE6F2A0E61
:1021FA00AF6F000EB06FA2DC0D0E0B6E2D0E0C6EC3
:10220A00D70E0D6E0D2EFED70C2EFCD70B2EFAD73D
:10221A00000000007C86020E7D6E700EAB6EA884F4
:10222A0061DC0C0EB86FA0EC0AF01F0E0B6E710E7B
:10223A000C6E1E0E0D6E0D2EFED70C2EFCD70B2E1D
:10224A00FAD70000B10E0101AE6F280EAF6F000E73
:10225A00B06F74DC000E0101AE6F050EAF6F400E59
:10226A00B06F050EB16FABEC0CF0D4DD9F0EAE6F04
:10227A00290EAF6F000EB06FC9DE6D0E0101AE6F91
:10228A00290EAF6F000EB06FC1DE8A0E0101AE6F6C
:10229A00270EAF6F000EB06FB9DEB30E0101AE6F3D
:1022AA00290EAF6F000EB06FB1DE0D0E0B6E2D0E44
:1022BA000C6ED70E0D6E0D2EFED70C2EFCD70B2EE4
:1022CA00FAD70000000022DF410EAE6F2A0EAF6F70
:1022DA00000EB06F33DCB8DE400E0101AE6F050EA2
:1022EA00AF6F070EB06F2A0EB16F000EB26FBEDE6F
:1022FA00400E0101B86F050EB96F400EBA6F7AEC45
:10230A000CF0005201E1F4D785DD400EAE6F050EE8
:10231A00AF6F310EB06F000EB16FD1DE400EB86FE5
:10232A00050EB96F400EBA6F7AEC0CF0005201E15B
:10233A00F5D7400EAE6F050EAF6F510EB06F000E9F
:10234A00B16FBDDE400EB86F050EB96F400EBA6FA1
:10235A007AEC0CF0005201E1F5D7070E0B6E170E5E
:10236A000C6E6A0E0D6E0D2EFED70C2EFCD70B2EA0
:10237A00FAD70000400EAE6F050EAF6F870EB06F32
:10238A00290EB16F000EB26F71DE400E0101B86FF7
:10239A00050EB96F400EBA6F7AEC0CF0005201E1EB
:1023AA00F4D755DD00C064F101C065F102C066F1E1
:1023BA0003C067F100C0AEF101C0AFF102C0B0F1D5
:1023CA0003C0B1F1550EB26F000EB36FEDEC0CF015
:1023DA00400EAE6F050EAF6F550EB06F000EB16FA7
:1023EA006EDE400EB86F050EB96F400EBA6F7AEC0A
:1023FA000CF0005201E1F5D70DDD650EAE6F280E27
:10240A00AF6F000EB06FA3EC0DF08B0E0101AE6F33
:10241A00280EAF6F000EB06FF9DD78DE64EC0DF0B8
:10242A009D8AA38AF28CF28E97EC0CF06D0E000155
:10243A00AD6F000EAE6FC50E0101AE6F290EAF6F04
:10244A00000EB06FE3DD000E83BE010E0101B86F0E
:10245A00300EB827A0EC0AF0710E0101AE6F2A0EF9
:10246A00AF6F000EB06FD2DD000E87B6010E01010C
:10247A00B86F300EB827A0EC0AF0DEDC0101AE6BB3
:10248A0042DD00C00DF101C00EF100C0AEF101C085
:10249A00AFF1550E0101B06F000EB16FE9DC790E94
:1024AA00AE6F2A0EAF6F000EB06FA3EC0DF0550E93
:1024BA000101AE6F000EAF6F5EDDD1DC000E0101CF
:1024CA000C1902E1010E0B1910E1330EAE6F2A0E40
:1024DA00AF6F000EB06FA3EC0DF00F0E0101AE6FDF
:1024EA00010EAF6F48DDBBDC11DE000E501802E1B1
:1024FA00010E4F1810E1250EAE6F2A0EAF6F000EB7
:10250A00B06F84DDAF0E0101AE6F000EAF6F11DE4A
:10251A0093DC64EC0DF028DE005207E1000E02198C
:10252A0002E1000E011901E1F6D7000E021902E1DB
:10253A00010E011903E197EC0CF0E9D0000EAE6F21
:10254A00050EAF6FFBDC00C05FF101C060F1ADC0EA
:10255A00AEF1AEC0AFF1000EB06F050EB16FAFDDD8
:10256A00400EAE6F050EAF6F160EB06F2A0EB16F2A
:10257A00000EB26F7BDD400E0101B86F050EB96F18
:10258A00400EBA6F7AEC0CF0005201E1F4D7400E1B
:10259A00AE6F050EAF6FADC0B0F1AEC0B1F18FDD59
:1025AA00400EB86F050EB96F400EBA6F7AEC0CF098
:1025BA00005201E1F5D72EDC000EAE6F050EAF6FAB
:1025CA00380EB06F000EB16F060EB26FEEDC000E61
:1025DA00011802E1000E001819E18C88400E010171
:1025EA00AE6F050EAF6F660EB06F2A0EB16F000E9A
:1025FA00B26F3CDD400E0101B86F050EB96F400E97
:10260A00BA6F7AEC0CF0005201E1F4D70101000E26
:10261A00AE6F050EAF6F300EB06F000EB16F070EC2
:10262A00B26FC3DC000E011802E1000E001819E1B6
:10263A008C98400E0101AE6F050EAF6FF80EB06FA9
:10264A00290EB16F000EB26F11DD400E0101B86F95
:10265A00050EB96F400EBA6F7AEC0CF0005201E128
:10266A00F4D70101000EAE6F050EAF6F290EB06FE1
:10267A00000EB16F060EB26F98DC000E011802E16F
:10268A00000E001819E18D88400E0101AE6F050E8B
:10269A00AF6F5B0EB06F2A0EB16F000EB26FE6DC41
:1026AA00400E0101B86F050EB96F400EBA6F7AEC91
:1026BA000CF0005201E1F4D70101000EAE6F050ED5
:1026CA00AF6F3F0EB06F000EB16F070EB26F6DDCC9
:1026DA00000E011802E1000E001819E18D98400E53
:1026EA000101AE6F050EAF6FE90EB06F290EB16F23
:1026FA00000EB26FBBDC400E0101B86F050EB96F58
:10270A00400EBA6F7AEC0CF0005201E1F4D78ED683
:02271A00FFD7E7
:102A840010EE29F01E0E006E010E016E1B0EF66E86
:0E2A9400290EF76E000EF86E5CEC0DF01200CD
:10271C0031384638374A353020436C69636B657203
:10272C00323A20546573742055415254312C554122
:10273C005254322C4849442C54696D6572302C41EA
:08274C00444330200D0A200077
:1027540050726F6A65743A205049433138463837AD
:102764004A35305F55415254315F55415254325FBE
:102774004849445F414443305F746573742E6D630C
:062784007070690D0A00EF
:10278A002055415254322026204144432054657337
:10279A007473207769746820436C69636B6572325D
:0F27AA002050494331384638374A35300D0A0040
:1027B90020554152543120205465737420414443BB
:1027C90030207769746820436C69636B65723220C5
:0E27D90050494331384638374A35300D0A0032
:1027E7002A035000490043003100380046003800F2
:1027F70037004A0035003000200043006C006900B4
:0E28070063006B0065007200320000000000EC
:1028150009022900010100803209040000020300B9
:102825000000092101010001222100070581034063
:0928350000010705010340000148
:10283E005541525420434F4D313A31393230302CBC
:10284E0020554152543220434F4D3232203A3139C5
:07285E00333030200D0A00A9
:102865002041726D65204954205541525431202E26
:102875002E20426F75636C65207072696E63697096
:06288500616C650D0A0004
:10288B002041726D65204954205541525432202EFF
:10289B002E2E426F75636C65207072696E63697062
:0628AB00616C650D0A00DE
:1028B100417474656E746520496E6974206C696138
:1028C10069736F6E20484944205465726D696E6169
:0528D1006C200D0A005F
:1028D6002403530061006200650072002000450079
:1028E6006C0065006300740072006F006E00690082
:0428F6006300730008
:1028FA000600FF0901A10119012940150026FF0060
:10290A007508954081021901294075089540910280
:01291A00C0FC
:07291B004C44325F4F4E00F7
:082922004C44315F4F464600B2
:07292A004C44315F4F4E00E9
:082931004C44325F4F464600A2
:102939002056657273696F6E203A2032392D30370F
:0A2949002D3230313520610D0A00F7
:10295300513D384D485A207820504C4C203D3E2064
:0A29630034384D487A20200D0A0098
:10296D002056657273696F6E203A2032392D3037DB
:0A297D002D3230313520610D0A00C3
:1029870020466F736320284B687A29206176656338
:0829970020504C4C3D312000A2
:10299F0020496E6974204849442055534220636F83
:0429AF006D0D0A00A0
:1029B30020496E69742054696D6572302049540D45
:0229C3000A0008
:1029C5002045746174206465200920204250313D02
:0229D5002000E0
:1029D7001201000200000008341201000100010288
:0229E7000001ED
:0F29E90053687574646F776E204C44320D0A008A
:0F29F80053687574646F776E204C44310D0A007C
:0F2A070032392D30372D3230313520610D0A0034
:0F2A1600526563657074696F6E2064653A2000C5
:0E2A250055415254322052656375203A20000C
:0E2A330055415254312052656375203A2000FF
:0D2A410020496E697420414443300D0A00A5
:0D2A4E0020496E697420414443300D0A0098
:0B2A5B0046697265204C44320D0A00F1
:0B2A660046697265204C44310D0A00E7
:082A710020425032203D2000FC
:062A790045414F3D200025
:042A7F00040309043F
:020000040001F9
:06FFF800ACF7C5FFF8FFA5
:00000001FF
